:10000000AE29FF3FFF3FFF3F0030031383129F1BCA
:100010000130F1007108013A031D12280130A000DF
:10002000851113288515080003138312A101A2016D
:100030002F082202031D1E282E082102031824283F
:10004000A10A0319A20A18280800353400343B34E9
:1000500000342F340034413400342A340034463420
:100060000034243400344C3400341F340034513410
:1000700000341A34003456340034153400345B3400
:100080000034113400345F3400340D3400346234F1
:1000900000340934003466340034063400346834E3
:1000A0000034043400346B340034023400346C34D3
:1000B0000034003400346D340034003400346E34C5
:1000C0000034003400346E340034003400346D34B5
:1000D0000034013400346C340034033400346A34A6
:1000E0000034053400346734003408340034643498
:1000F00000340B340034613400340F3400345D3488
:10010000003413340034583400341734003453347A
:1001100000341C3400344E3400342234003449346A
:10012000003427340034443400342D3400343E3459
:10013000003432340034383400343834003432344B
:1001400000343E3400342D34003444340034273439
:10015000003449340034223400344E3400341C342A
:10016000003453340034173400345834003413341A
:1001700000345D3400340F340034613400340B3407
:1001800000346434003408340034673400340534F7
:1001900000346A340034033400346C3400340134E5
:1001A00000346D340034003400346E3400340034D4
:1001B00000346E340034003400346D3400340034C4
:1001C00000346C340034023400346B3400340434B2
:1001D00000346834003406340034663400340934A2
:1001E0000034623400340D3400345F340034113490
:1001F00000345B34003415340034563400341A347F
:100200000034513400341F3400344C34003424346E
:100210000034463400342A340034413400342F345E
:1002200000343B34003435340034080003138312A7
:1002300024088A002508820008008B13033003136A
:1002400083168600831286019F129F151F119F142B
:100250001F10E430831685008312851583169F17BF
:100260001F139F129F151F119F101F1408000313C7
:100270008312A0011E30A6000030A700A801A9012A
:10028000AA01080003138312AB0100302706031DE7
:100290004B2926082B06031D4E290420061786121B
:1002A0000130F4002B08F000F101740803195D29F6
:1002B000F00DF10D7010FF3F56292530F00700308A
:1002C0000318013FF1077008A5007108A4000A088F
:1002D000A3001621AE0023088A00A50A0319A40A68
:1002E0001621AF0023088A001420AB0A06138616D5
:1002F0000130F4002B08F000F1017408031985297E
:10030000F00DF10D7010FF3F7E292530F007003011
:100310000318013FF1077008A5007108A4000A083E
:10032000A3001621AE0023088A00A50A0319A40A17
:100330001621AF0023088A001420AB0A2D08003CC8
:10034000031DA4292C082B02031C45290800783022
:1003500003138312AC000030AD000800A7211D215B
:1003600037214221A90A0319AA0A00302A06031DCF
:10037000BB2932302906031DCF29A901AA01C729AB
:100380000130A8008617CF29A8018613CF29280895
:10039000003A0319C0292808013A0319C429B129D0
:1003A000D029FF3FFF3FFF3FFF3FFF3FFF3FFF3FA2
:02400E006A3F07
:00000001FF
